:020000040000FA
:04000000A0EF7FF0FE
:08FF38000000000000000000C1
:10FF400082B2FAD7240EAC6E0A0EAF6E900EAB6E74
:10FF500046D8C10853E14F0EAD6E4B0EAD6E006A30
:10FF60003ED8F86E076E3BD8F76EA96E38D8F66E9D
:10FF7000A86E35D8016E012A00EE09F0F56E2FD873
:10FF8000EC6E012EFBD700661FD007AC03D0040E29
:10FF90001ED818D007AE04D00C00C40E18D812D04A
:10FFA000940E15D80A00080E056E00EE0AF0080E31
:10FFB000066EEE50F56E0F00062EFBD7840E07D8A6
:10FFC000052EF5D7A694C9D74E0EAD6EC8D7A66E2E
:10FFD000550EA76EAA0EA76EA68200001200370E5D
:10FFE000026E036A046A9EAA03D0AE500026120075
:10FFF000042EF9D7032EF6D7022EF3D7AB9E9CD74B
:020000040030CA
:0300010002161EC6
:020005008081F8
:060008000FC00FE00F40E5
:00000001FF
